:1064FA000A2A2A2A2A2A2A2A2A2A2A2A2A2A2A2A12
:10650A002A2A20CFE0F0E0ECE5F2F0FB20E0E4E01C
:10651A00EFF2E5F0E0202A2A2A2A2A2A2A2A2A2A17
:10652A002A2A2A2A2A2A2A2A0A00312E204D4143B7
:10653A0020E0E4F0E5F13A202025303262783A256D
:10654A00303262783A25303262783A2530326278CF
:10655A003A25303262783A25303262780A00322E91
:10656A0020495020E0E4F0E5F13A20202025627528
:10657A002E2562752E2562752E2562750A00332E28
:10658A0020D8EBFEE73A2020202020202025627523
:10659A002E2562752E2562752E2562750A00342E07
:1065AA0020CCE0F1EAE020F1E5F2E83A2025627534
:1065BA002E2562752E2562752E2562750A00352EE6
:1065CA0020495020E0E4F0E5F120F1E5F0E2E5F0C1
:1065DA00E0313A202562752E2562752E2562752EC8
:1065EA002562750A00362E20495020E0E4F0E5F1D4
:1065FA0020F1E5F0E2E5F0E0323A202562752E2539
:10660A0062752E2562752E2562750A00372E20D2F4
:10661A00E0E9EC2DE0F3F220EEF2E2E5F2E020F11F
:10662A00E5F0E2E5F0E03A2025627520282A3130CB
:10663A006D63290A00302E20CAEBFEF720E4EEF142
:10664A00F2F3EFE03A2025730A000AC7C0CFC8D197
:10665A00DC20466C6173680A000AC7E0EFE8F1FCC7
:10666A0020E7E0E2E5F0F8E5EDE0210A000820087D
:10667A00000A53696E636F6D4950205665722E2069
:10668A00322E3020434320282770272DE2F5EEE4EE
:10669A0020E220EAEEEDF4E8E3F3F0E0F2EEF0298E
:1066AA00000A3E20CAEEEDF4E8E3F3F0E0F6E8EE85
:1066BA00EDEDFBE920F0E5E6E8EC0A0A00203C49AA
:1066CA003E20203A20CFEEEAE0E7E0F2FC20EFE0BD
:1066DA00F0E0ECE5F2F0FB0A00203C536E3E203A73
:1066EA0020C7E0E4E0F2FC20EFE0F0E0ECE5F2F0B5
:1066FA0020276E270A00203C4B3E20203A20C7E084
:10670A00E3F0F3E7E8F2FC20EDEEE2F3FE20EAEE36
:10671A00EDF42E20E8E720F4E0E9EBE00A00203C63
:10672A00443E20203A20D0E0F1EFE5F7E0F2E0F233
:10673A00FC20EDEEE2F3FE20EAEEEDF42E0A002054
:10674A003C573E20203A20C7E0EFE8F1E0F2FC2077
:10675A00E8E7ECE5EDE5EDE8FF0A00203C4C3E20D9
:10676A00203A20C7E0E3F0F3E7E8F2FC20EFF0EE8E
:10677A00E3F0E0ECECF30A00203C453E20203A200E
:10678A00C2FBF5EEE40A003E20C2E2E5E4E8F2E5E7
:10679A0020EAEEECE0EDE4F33A20000AC2E2E5E496
:1067AA00E8F2E520274D414320E0E4F0E5F15B25DE
:1067BA0062645D273A202530326278202D3E0078C7
:1067CA00000AC2E2E5E4E8F2E52027495020E0E4C5
:1067DA00E0EFF2E5F0E05B2562645D273A2025628E
:1067EA0075202D3E0075000AC2E2E5E4E8F2E520D4
:1067FA0027D8EBFEE75B2562645D273A20256275A0
:10680A00202D3E000AC2E2E5E4E8F2E52027CCE0CA
:10681A00F1EAF3D1E5F2E85B2562645D273A2025C7
:10682A006275202D3E000AC2E2E5E4E8F2E520277F
:10683A00495020F1E5F0E2E5F0E0315B2562645D64
:10684A00273A20256275202D3E000AC2E2E5E4E8D7
:10685A00F2E52027495020F1E5F0E2E5F0E0325B6D
:10686A002562645D273A20256275202D3E000AC202
:10687A00E2E5E4E8F2E52027C2F0E5ECFF20EEE6E7
:10688A00E8E4E0EDE8FF20EEF2E2E5F2E0273A2064
:10689A00256275202D3E000AC2E2E5E4E8F2E52011
:1068AA00EAEBFEF720E4EEF1F2F3EFE028E4EE2063
:1068BA003720F1E8ECE2293A0A2D3E000A20457217
:1068CA00726F72210A000AC8C4C5D220C7C0CFC8D5
:1068DA00D1DC2120C6C4C8D2C521000AC7C0CFC88E
:1068EA00D1DC20C7C0C2C5D0D8C5CDC0210A000A94
:1068FA0020000ACA20EFF0E8E5ECF320E3EEF2EE1E
:10690A00E2210A000ACEF8E8E1EAE020E7E0E3F053
:10691A00F3E7EAE8210A000AD4E0E9EB20EFEEEB1C
:10692A00F3F7E5ED210A00CEF8E8E1EAE0210A00F2
:10693A000AD4E0E9EB20EFEEEBF3F7E5ED2120C70F
:10694A00E0EFE8F1FC20E220454550524F4D210A84
:10695A00003C4D41433D003C4130313D003C41301B
:10696A00323D003C4130333D003C4130343D003C37
:10697A004130353D003C4130363D000ACAEEEDF467
:10698A00E8E3F3F0E0F6E8FF20E7E0EFE8F1E0ED16
:04699A00E0210A00EE
:10767B00C2ADE4F5C9D2CDD2CCC2C9C2CAF5CDF5E3
:10768B00CC75CBFF75CAB885CBCD85CACCD29ED273
:10769B009CD2CAE59924FF92CAC2ACC298C2993057
:0676AB0099032098FA2269
:07780C003098FDAF99C2980E
:017813002252
:0677F20012780CEFF522F5
:0877F8008F993099FDC299221E
:1077E200AE07BE0A057F0D1277F8AF061277F822B0
:1072C6007BFF7A6479FA126A007BFF7A65793490DB
:1072D60060A2E0F537A3E0F538A3E0F539A3E0F5C1
:1072E6003AA3E0F53BA3E0F53C126A007BFF7A6522
:1072F60079689060A8E0F537A3E0F538A3E0F539A2
:10730600A3E0F53A126A007BFF7A65798890609A65
:10731600E0F537A3E0F538A3E0F539A3E0F53A1236
:107326006A007BFF7A6579A890609EE0F537A3E056
:10733600F538A3E0F539A3E0F53A126A007BFF7A47
:107346006579C89060B1E0F537A3E0F538A3E0F5BC
:1073560039A3E0F53A126A007BFF7A6579EF90600F
:10736600B5E0F537A3E0F538A3E0F539A3E0F53A43
:10737600126A007BFF7A6679169060B9E0F53712DB
:107386006A007537017538607539CB7BFF7A667987
:047396003F026A0048
:067467008E2B8F2C8D2DF1
:10746D00E4F532F533F530F531E52D60097BFF7A22
:10747D00667954126A00E4F52EF52FE52BC4F85405
:10748D00F0C868FEE52CC4540F48FFC3E52F9FE5F7
:10749D002E9E5040AE32AF33AD07AC067B10AF31F0
:1074AD00AE3012771A74102533F533E43532F532D8
:1074BD0074102531F531E43530F530E52D600BE5EF
:1074CD002F543F70057F231277F8052FE52F70ABF2
:1074DD00052E80A7E52BC4F854F0C868FEE52CC432
:1074ED00540F48C4F8540FC868FFEEC454F048FE5A
:1074FD00C3E52C9FFFE52B9EAC32AD33AB07AF310F
:10750D00AE3012771AE52D60097BFF7A667963122A
:02751D006A0002
:01751F002249
:04739A007E677FEF9C
:04739E008E298F2A7B
:1073A200E4F52B7400252BF582E43460F583E4F0D8
:1073B200052BE52BB408ECE4F52B12780CEFF52C39
:1073C200640A6005E52CB40D0F7400252BF582E4E8
:1073D2003460F583E4F08044E52CB40824E52BD333
:1073E2009400402F7BFF7A667977126A00152B741E
:1073F20000252BF582E43460F5837420F0152B8090
:10740200127400252BF582E43460F583E52CF0FF3D
:107412001277F8052BE52BC39408409EE52B7002EA
:10742200FF22852A82852983E493B4781E90600026
:10743200E0FF1276E6EFC454F0FEC006906001E071
:10744200FF1276E6D0E02FF508801775310075320D
:1074520000753300E4F5347B017A60790012712201
:047462008F087F010F
:017466002203
:10600300752501C2AF907FFEE0B4FF047F018002DB
:106013007F00907FFDE0B4AA047E0180027E00EE43
:106023005FFF907FFFE0B455047E0180027E00EEA7
:106033005F6028E4907FFDF0A3F0A3F0907FF0E091
:10604300FEA3E0FF4E6005E4FD1274677BFF7A0058
:1060530079008B268A278928126FED12767BC298E6
:106063007BFF7A66797B126A0030980F7BFF7A0098
:1060730079008B268A278928126FEDE4F523E4F54E
:10608300242098030264C512780CEFF52264506053
:1060930009E522647060030264B6AF221277F87FC9
:1060A3000A1277F8E4F523E5232401FFE433FE1213
:1060B300776D749A2523F582E43460F583EFF00558
:1060C30023E523C3943F40DFE4F523E523247FFF47
:1060D300E433FE12776D74142523F582E43460F5FE
:1060E30083EFF00523E523C3948040DFE4906093BE
:1060F300F0E52570030264C57BFF7A6679AB126A0B
:10610300007BFF7A6679C7126A007BFF7A6679E3C0
:10611300126A007BFF7A677900126A007BFF7A6755
:106123007928126A007BFF7A677949126A007BFF3C
:106133007A677965126A007BFF7A677982126A004F
:106143007BFF7A677991126A001277F2E522126F68
:10615300C7646F4464004561824964694B64634C5E
:10616300618853640657646F64640065618269647F
:10617300696B64636C618873640677000060F41272
:1061830072C60260F41277F2E522126FC7634B30D6
:1061930061AC3161EF32622E33626D3462AC3562D1
:1061A300EB36632A37000063F8E4F522E522C39453
:1061B3000640030260F47BFF7A6779A58522377472
:1061C300A22522F582E43460F583E0F538126A00F3
:1061D3007E677FC912739EEF600E74A22522F5823B
:1061E300E43460F583E508F0052280C0E4F522E598
:1061F30022C3940440030260F47BFF7A6779CB8562
:10620300223774A82522F582E43460F583E0F5385B
:10621300126A0012739AEF600E74A82522F582E4C5
:106223003460F583E508F0052280C4E4F522E52215
:10623300C3940440030260F47BFF7A6779F18522FB
:1062430037749A2522F582E43460F583E0F5381239
:106253006A0012739AEF600E749A2522F582E43471
:1062630060F583E508F0052280C4E4F522E522C346
:10627300940440030260F47BFF7A68790E85223729
:10628300749E2522F582E43460F583E0F538126AC2
:106293000012739AEF600E749E2522F582E4346037
:1062A300F583E508F0052280C4E4F522E522C394D2
:1062B3000440030260F47BFF7A68793085223774E7
:1062C300B12522F582E43460F583E0F538126A00E3
:1062D30012739AEF600E74B12522F582E43460F5EF
:1062E30083E508F0052280C4E4F522E522C3940483
:1062F30040030260F47BFF7A68795485223774B5D2
:106303002522F582E43460F583E0F538126A001241
:10631300739AEF600E74B52522F582E43460F58339
:10632300E508F0052280C47BFF7A6879789060B92C
:10633300E0F537126A0012739AEF70030260F4906B
:1063430060B9E508F00260F47BFF7A6879A1126A0C
:1063530000E4F52374CB2523F582E43460F583E46C
:10636300F00523E523B408ECE4F52312780CEFF5EC
:1063730022640A6005E522B40D0F74CB2523F58250
:10638300E43460F583E4F08044E522B40824E52393
:10639300D39400402F7BFF7A667977126A00152326
:1063A30074CB2523F582E43460F5837420F0152340
:1063B300801274CB2523F582E43460F583E522F063
:1063C300FF1277F80523E523C39408409E9060CB22
:1063D300E0642060030260F4F523E523C3940840DE
:1063E300030260F474CB2523F582E43460F583E47F
:1063F300F0052380E57BFF7A6879C6805DE4F525A7
:106403000260F47BFF7A6879D0126A00E4F523E531
:10641300232401FFE433FE749A2523F582E43460D8
:10642300F583E0FD1277890523E523C3943F40DF1D
:10643300E4F523E523247FFFE433FE74142523F5D9
:1064430082E43460F583E0FD1277890523E523C3F5
:10645300948040DF7BFF7A6879E5126A000260F47A
:106463001276B10260F4126CFA0260F47BFF7A6870
:1064730079F9126A00906094E4F0A374FFF0E4F5F4
:1064830023C3E52394D07480948740030260F4E52A
:1064930022F470030260F4E52270030260F41277C1
:1064A300BA8F221277F8E522642170030260F405A3
:1064B3002380CE7BFF7A0079008B268A27892812D6
:1064C3006FED7F057E0012774E0524E524C39419F2
:1064D30050030260847F2E1277F80523E523C394CB
:1064E3000A50030260817BFF7A0079008B268A279A
:0764F3008928126FED80FE05
:10774E00E4FDFCC3ED9FEC9E5014E4FBFA0BBB0072
:0E775E00010AEBF44A70F60DBD00010C80E547
:01776C0022FA
:107520009060D9126F9600000000E4F52BF52C2036
:10753000983CD3E52C9400E52B940040199060D939
:10754000126F72EF2401FFE43EFEE43DFDE43CFCDB
:107550009060D9126F8AE47FE87E03FDFC9060D9C9
:10756000126F7ED3126F6140C6AE2BAF2C2290609B
:10757000D9126F960000000012780C852C82852BA2
:1075800083EFF0E52B5403452C70057F2A1277F822
:10759000052CE52C7002052BC394C0E52B945D40AF
:0575A0008E7E007F015A
:0175A50022C3
:1076B1007BFF7A6879FC126A001275208E298F2A65
:1076C100C3E52A94E8E52994037BFF50077A697999
:1076D1000E026A007A697921126A007D01AF2AAE31
:0476E100291274678F
:0176E5002282
:1076E600EFC39430400BEFD394395005EF24D0FF0D
:1076F60022EFC39461400BEFD394665005EF24A9A3
:10770600FF22EFC39441400BEFD394465005EF247C
:04771600C9FF222263
:1077BA00906094E475F001126F4B906094E0FEA320
:0677CA00E0FF12776D22C2
:1077A2001277BA1276E6EFC454F0FEC0061277BA28
:0877B2001276E6D0E02FFF2261
:107626001277BA906000EFF01277BA906001EFF02F
:107636001277BA906002EFF01277BA906003EFF01B
:107646001277BA906004EFF01277BA906005EFF007
:107656001277BA906006EFF01277BA906007EFF0F3
:10766600E4A3F0F531F532F533F5347B017A607930
:05767600001271222248
:0475A6008E2E8F2F67
:1075AA00906094E4F0A374FFF01277BAEF6069F484
:1075BA006066852F82852E83E493B507EC753001CA
:1075CA00E52F2530F582E4352EF583E49360259086
:1075DA006095E02530FF906094E03400FE12776DEC
:1075EA00E52F2530F582E4352EF583E493B50704BB
:1075FA00053080CCE52F2530F582E4352EF583E47D
:10760A009370A6E53024FFFFE434FF9060948FF076
:0B761A00126F4B7E007F0122E4FEFF98
:017625002242
:106CFA007BFF7A6879FC126A009060D9126F96005D
:106D0A00000000E4F529F52A209841D3E52A9400E9
:106D1A00E529940040199060D9126F72EF2401FF9F
:106D2A00E43EFEE43DFDE43CFC9060D9126F8A7FAC
:106D3A00E07E937D047C009060D9126F7ED3126F3F
:106D4A006140C57BFF7A697931026F479060D91239
:106D5A006F960000000012780C8F2DE52D643C60C0
:106D6A0011052AE52A70020529C394C0E529945D14
:106D7A004096900000E52DF0752900752A011278D9
:106D8A000C8F2D852A82852983E52DF064216011D7
:106D9A00052AE52A70020529C394D0E529940740FB
:106DAA00DD7BFF7A69793A126A00E52A2401F52C1B
:106DBA00E43529F52BE4F529F52AC3E52A952CE5CE
:106DCA0029952B501EE4252AFFE5293401FE852A40
:106DDA0082852983E0FD127789052AE52A70DB0579
:106DEA002980D77E697F5B1275A6EF4E60301277D5
:106DFA00A29060A2EFF01277A29060A3EFF0127750
:106E0A00A29060A4EFF01277A29060A5EFF012773B
:106E1A00A29060A6EFF01277A29060A7EFF07E69C9
:106E2A007F611275A6EF4E60201277A29060A8EFDC
:106E3A00F01277A29060A9EFF01277A29060AAEF01
:106E4A00F01277A29060ABEFF07E697F671275A6A9
:106E5A00EF4E60201277A29060B1EFF01277A29005
:106E6A0060B2EFF01277A29060B3EFF01277A290BF
:106E7A0060B4EFF07E697F6D1275A6EF4E60201246
:106E8A0077A29060B5EFF01277A29060B6EFF01299
:106E9A0077A29060B7EFF01277A29060B8EFF07E19
:106EAA00697F731275A6EF4E60201277A290609EDA
:106EBA00EFF01277A290609FEFF01277A29060A095
:106ECA00EFF01277A29060A1EFF07E697F791275D8
:106EDA00A6EF4E60201277A290609AEFF01277A286
:106EEA0090609BEFF01277A290609CEFF01277A26D
:106EFA0090609DEFF07E697F7F1275A6EF4E600865
:106F0A001276269060B9EFF0E4F529F52AE52A24ED
:106F1A0001FFE43529FE749A252AF582E43460F5E6
:106F2A0083E0FD127789052AE52A70020529C394B0
:106F3A0043E529940040D67BFF7A697985126A0075
:016F4A002224
:02771A008B34AE
:10771C00A2AF9200C2AF85A23553A2FE8E838F8298
:10772C0005A28C838D8274091277D0E53453A2FEA6
:10773C0043A2201277D253A2DF8535A2A20092AFCA
:01774C00FF3D
:01774D002219
:10776D00E5D220E0FBC2AF438E2075D2028F828E10
:0B777D0083E0FFE4F5D2538EDFD2AFB3
:0177880022DE
:10778900E5D220E0FBC2AF43D2028F828E83EDF0B7
:0977990075D25063D250D2AF2228
:1077D000F922C002C004C00612FFF0D006D004D0C7
:0277E000022283
:0360000002780023
:0C78000078FFE4F6D8FD758147026003B4
:106F4B00C5F0F8A3E028F0C5F0F8E58215827002D1
:066F5B001583E038F0226E
:106F6100EB9FF5F0EA9E42F0E99D42F0E89C45F086
:016F710022FD
:0C6F7200E0FCA3E0FDA3E0FEA3E0FF2292
:0C6F7E00E0F8A3E0F9A3E0FAA3E0FB2296
:0C6F8A00ECF0A3EDF0A3EEF0A3EFF0227A
:106F9600A8828583F0D083D082126FAD126FAD12B6
:106FA6006FAD126FADE473E493A3C583C5F0C583DB
:106FB600C8C582C8F0A3C583C5F0C583C8C582C845
:016FC60022A8
:106FC700D083D082F8E4937012740193700DA3A359
:106FD70093F8740193F5828883E47374029368606D
:066FE700EFA3A3A380DF6D
:066FED008A838982E4732F
:10699E00E5432437F8E6054322783430070278378A
:1069AE00E475F0011270A8026FF32000EB7F2ED277
:1069BE00008018EF540F2490D43440D4FF30040BD1
:1069CE00EF24BFB41A0050032461FFE544600215A2
:1069DE00440547E5477002054630070D7834E475E7
:1069EE00F0011270A8EF0270390277E27403D20739
:1069FE008003E4C207F5438B348A358936E4F544C7
:106A0E00F546F547E54460077F201269D980F57594
:106A1E0045FFC201C200C202C203C205C206C208BD
:106A2E001269A7FF700D3007057F001269EAAF47A4
:106A3E00AE4622B4255FC2D5C2041269A7FF24D088
:106A4E00B40A00501A75F00A784430D50508B6FF1E
:106A5E000106C6A426F620D5047002D20380D924DE
:106A6E00CFB41A00EF5004C2E5D204026BEAD20191
:106A7E0080C6D20080C0D20280BCD2D580BAD205E8
:106A8E0080B47F201269D92002077401B5440040FA
:106A9E00F112699EFF1269D9026A12D208D20680DB
:106AAE009512699EFB12699EFA12699EF94A4B7005
:106ABE000679BB7A6C7BFF20022EE544602A7E00AD
:106ACE008E8275830012700C60060EEE654570F0B6
:106ADE00C2D5EBC0E0EAC0E0E9C0E0EE126C31D006
:106AEE00E0F9D0E0FAD0E0FB126FF3FF60AAEBC042
:106AFE00E0EAC0E0E9C0E01269D9D0E02401F9D0A3
:106B0E00E03400FAD0E0FBE5450460DCD545D980E1
:106B1E00877BFF7A6C792DD202809C791080027966
:106B2E0008C206C2088008D2D5790A8004790AC242
:106B3E00D5E545047002F545E4FAFDFEFF12699EA7
:106B4E00FC7B0820011312699EFD7B1030000A1297
:106B5E00699EFE12699EFF7B20EC3382D592D55042
:106B6E0013C3E43000069FFFE49EFEE42001039D64
:106B7E00FDE49CFCE4CBF8C201EC700CCFCECDCC86
:106B8E00E824F8F870F38017C3EF33FFEE33FEED11
:106B9E0033FDEC33FCEB33FB994002FB0FD8E9EBF2
:106BAE00300105F8D0E0C448B201C0E00AEC4D4E09
:106BBE004F78207B0070C2EAB5450040BCC0E012A1
:106BCE006C33D0F0D0E0200104C4C0E0C4B201C0E8
:106BDE00F01269C2D0F0D5F0EB026A12126FC76ADA
:106BEE00AF536B29586A804C6A7C426B2D4F6B35C4
:0F6BFE00446B35496A95436B3B556B1F466B1FC4
:106C0D00456B1F476CDB506A842D6A882E6AAB2B4F
:106C1D006A8C236AA9206CC42A6A444800006AA3BE
:106C2D003F3F3F00790AA2D5200314300509B91062
:106C3D00020404B9080104A2D52006025001042063
:106C4D0002689202B544005034C0E07F2030031931
:106C5D007F30A20272067205500F126C8AC202C2F8
:106C6D0006C205C2087F30800F300503E9C0E0126F
:106C7D0069D9300503D0E0F9D0E0B544CC30051723
:106C8D007F30B9100C1269D97F583004077F788096
:106C9D0003B908031269D93002057F2D0269D97F26
:106CAD00202008F87F2B2006F322920280CF286E39
:106CBD00756C6C2900D20112699E3001F8C2017801
:106CCD004430D50108F6026A442D504349581269E3
:106CDD009E2403B405004001E4906CD6931269CA5A
:0D6CED00743A1269CAD203754404026B297F
:107122008B2E8A2F8930E4F53AF539F538F537F5A3
:1071320035F536E532453345316012EBC0E0EAC041
:10714200E0E9C0E0AB31AA32A9331270B8AB2E0528
:1071520030E530AA2F7002052F14F9126FF3F53BB8
:10716200C394094007E53BD3940D40E1E53B64201D
:1071720060DBE53BB42D054336038016E53BB42BBB
:1071820005433601800C74FF2530F53074FF352F2E
:10719200F52FE53460046410703FAB2EAA2FA9309E
:1071A200126FF364306009E534702E75340A802959
:1071B20090000112700CFF64786004EFB45813431E
:1071C200360175341074022530F530E4352FF52F71
:1071D2008007E5347003753408AB2E0530E530AA1C
:1071E2002F7002052F14F9126FF3F53BC39461401F
:1071F2000AE53BD3947A5003533BDF74D0253BF529
:107202003BC3940A400CE53B9411406D74F9253B55
:10721200F53BE53BD395345060433601853A3F85D3
:10722200393E85383D85373CAF347E00E4FCFDAB0A
:107232003AAA39A938A83712704BC8ECC8C9EDC9A7
:10724200CAEECACBEFCBE4FCFDFEEB253BF53AEEF2
:107252003AF539ED39F538EC38F537AF3AAE39ADA4
:1072620038FCAB3FAA3EA93DA83CD3126F61500344
:107272000271DB4336040271DBE53620E003E48071
:107282002DE53245334531601EAB2EE53024FFF942
:10729200E52F34FFFAEBC0E0EAC0E0E9C0E0AB3131
:1072A200AA32A9331270B8E53630E20774FFFFFE46
:1072B200FDFC22E536AF3AAE39AD38AC3730E103EA
:0472C20002709A229A
:106FF300BB010689828A83E0225002E722BBFE029C
:09700300E32289828A83E49322CE
:10700C00BB010CE58229F582E5833AF583E0225039
:10701C0006E92582F8E622BBFE06E92582F8E22283
:0D702C00E58229F582E5833AF583E493229D
:10703900BB010689828A83F0225002F722BBFE0136
:02704900F32230
:10704B00E88FF0A4CC8BF0A42CFCE98EF0A42CFCE4
:10705B008AF0EDA42CFCEA8EF0A4CDA8F08BF0A462
:10706B002DCC3825F0FDE98FF0A42CCD35F0FCEBC1
:10707B008EF0A4FEA9F0EB8FF0A4CFC5F02ECD3986
:0F708B00FEE43CFCEAA42DCE35F0FDE43CFC22F3
:0E709A00C3E49FFFE49EFEE49DFDE49CFC2207
:1070A800FAE6FB0808E6F925F0F618E6CA3AF622E9
:1070B800BB011A89828A83D0F0D0E0F8D0E0F9D0F9
:1070C800E0FAD0E0FBE8C0E0C0F00271105016E929
:1070D800F8D083D082D0E0F9D0E0FAD0E0FBC082CB
:1070E800C083027107BBFE16E9F8D083D082D0E0D6
:0F70F800F9D0E0FAD0E0FBC082C0830271192208
:09710700EBF608EAF608E9F622AD
:09711000EBF0A3EAF0A3E9F02280
:09711900EBF208EAF208E9F222A7
:00000001FF
